:100000000C943C010C9459010C9459010C94590125
:100010000C9459010C9474010C945B010C946D01C7
:100020000C9459010C9459010C9459010C945901E8
:100030000C9459010C9459010C9459010C945901D8
:100040000C9459010C9459010C9459010C945901C8
:100050000C945901010F020F040F080F100F008FAD
:10006000004F002F001F00000100020003000400E9
:1000700005000600070009000A000B000C000D0037
:100080000F001000110013001400150017001800D5
:100090001A001B001D001F00200022002300250065
:1000A000270029002B002C002E00300032003400E5
:1000B000360038003B003D003F0041004400460050
:1000C00048004B004D0050005300550058005B00A5
:1000D0005E006000630066006A006D0070007300DF
:1000E00076007A007D008100850088008C009000F9
:1000F000940098009C00A000A400A900AD00B100ED
:10010000B600BB00C000C400C900CE00D400D900B6
:10011000DE00E400E900EF00F500FB00010107014B
:100120000E0114011B01210128012F0136013E019E
:1001300045014D0155015C0165016D0175017E01AF
:1001400086018F019801A201AB01B501BF01C90170
:10015000D301DE01E801F301FE010A0215022102CA
:100160002D0239024602530260026D027B028802B0
:100170009702A502B402C302D202E202F202020313
:10018000130324033503460358036B037E039103D3
:10019000A403B803CC03E103F6030C0422043804DF
:1001A0004F0467047E049704B004C904E304FD040B
:1001B000180533054F056C058905A705C505E40538
:1001C00004062406450666068806AB06CF06F30637
:1001D00018073E0765078C07B407DD0707083208D4
:1001E0005D088A08B708E508150945097609A809D0
:1001F000DB090F0A440A7B0AB20AEB0A240B5F0BE5
:100200009B0BD80B170C570C980CDA0C1E0D630DBA
:10021000A90DF10D3A0E850ED20E200F6F0FC00FF3
:1002200013106710BD1015116F11CB112812871212
:10023000E8124B13B11318148114EC145A15CA1593
:100240003C16B0162717A0171C189A181B199E19D0
:10025000241AAD1A381BC61B581CEC1C831D1D1E0E
:10026000BA1E5B1FFF1FFFFF00FF8000FF0000FFA3
:1002700000FF0000FF00FF0011241FBECFE5D4E007
:10028000DEBFCDBF10E0A0E6B0E0EAE3F8E002C0D8
:1002900005900D92A436B107D9F711E0A4E6B0E0BD
:1002A00001C01D92AB34B107E1F70E94B1030C9479
:1002B0001B040C9400007894CF93DF93E101299004
:1002C0003990499028BA32BA45BA2F8438883BBC55
:1002D0002ABC1E01DF91CF91189578940F920FB62A
:1002E00097D00FBE0F9018957894CF93DF930000AE
:1002F000DFEFC0EFD8BBD2BBC5BBC4E625BA3BBA63
:1003000048BA52BA65BAD0E02A803D804E8425BAF8
:1003100035BA000045BA0000288822BA00002884B7
:10032000398848805E806F8025BA2B8028BA35BA1C
:1003300048BA58BA0000298428BA00002C843980B1
:100340004C8028BA000032BA42BA000062BA2A844D
:10035000C6E722BA29903990499028BA32BA45BAEC
:100360001E01DF91CF911895ED91F0914601EF9F1D
:10037000F7FD1394F2E01F9EE6E6F0E0E00DF11DBC
:10038000059015900895F0DF06942794069437940D
:100390000694479406945794069467940694879419
:1003A000069497940694A7941694B7941694C794B9
:1003B0001694D7941694E7941694F79408952224EB
:1003C000332444245524662488249924AA24BB2455
:1003D000CC24DD24EE24FF2408952024302440245E
:1003E0005024602480249024A024B024C024D0244D
:1003F000E024F02428823B824E8259866C868F86C8
:100400009A8AAD8AB88ECB8EDE8EE9A2FCA20895C0
:100410000F921F92AF93BF93CF93DF93EF93FF930E
:100420008F929F92AF92BF92CF92DF92EF92FF9204
:100430007394E9E07E1608F07724A3EAB0E0E3E0E5
:100440007E9EA00DB11DE2E07E9EE4E5F0E0E00DB1
:10045000F11DC4E6D0E005900CAE05900DAEAFDF07
:1004600092DF91DF90DF58968EDF8DDF8CDF58961C
:100470008ADF89DF0A94B1DFA2DF85DF589684DF47
:1004800082DF81DF80DF58967EDF7DDF21960A9450
:10049000A4DF95DF78DF589676DF75DF74DF22946E
:1004A000329442945294629482949294A294B2941C
:1004B000C294D294E294F29421960BAC8EDF2297F0
:1004C0002DAC3CAC4F845D846B84FF90EF90DF904B
:1004D000CF90BF90AF909F908F90FF91EF91DF9161
:1004E000CF91BF91AF911F900F9008950024863354
:1004F00010F493E0899F83EA90E0800D911DFC0148
:100500000895F4DF4193519361930895EFDF819152
:100510009191A191BB270895FC01259135914491BA
:10052000B901CA010895269FB0011124489FC00156
:100530001124240F860F971F622F70E00E94F4038E
:10054000862F08958F929F92AF92BF92CF92DF92A3
:10055000EF92FF920F931F93DF93CF93CDB7DEB748
:1005600067970FB6F894DEBF0FBECDBF26E632E028
:10057000F90185919591A4918D839E83AF83B8876E
:10058000A9014D5F5F4F5A8749871C861B868B8563
:100590009C859B8B8A8BDE011196FE01359683E04C
:1005A00001900D928150E1F7E985FA85859095904B
:1005B000A4908D829E82AF82B88629813A814B8138
:1005C0005C812C8B3D8B4E8B5F8BBB27A52F942F93
:1005D000832F898BBB27AB2D9A2D892D888BCA0140
:1005E000AA27BB278F87C501AA27BB278E873AE09A
:1005F0003D87DA884B85D41A8C89682D4D852D2D41
:100600000E949302E82E898968894D852D2D0E94CC
:100610009302C82E8F856E854D852D2D0E949302E5
:10062000DC2CCC24FF24EC28FD280027F7FC0095C7
:10063000102F90E0A0E0B0E0DC0199278827E82A9D
:10064000F92A0A2B1B2B8A89B801A7010E94810273
:100650008A899B8901969B8B8A8B9D8591509D876A
:100660009F3F39F6AB85BC851A96BC87AB87298539
:100670003A852D5F3F4F3A872987DC9709F087CF6E
:1006800067960FB6F894DEBF0FBECDBFCF91DF9156
:100690001F910F91FF90EF90DF90CF90BF90AF90A0
:1006A0009F908F900895349B13C087B190E085563A
:1006B000904025B1FC01EA5BFE4F20830196833018
:1006C000910514F080E090E08B5987B987ED86B9E9
:1006D000909149019F5F90934901992321F0809166
:1006E00047018917E8F51092490140916000509147
:1006F0006100609162007091630080914A010E94E4
:10070000810280914A0180FD02C090E001C09FEF0C
:100710009093A3008F5F80934A01863309F581E0AF
:1007200080934A012091480180916000909161007E
:10073000A0916200B0916300820F911DA11DB11DB7
:1007400020E030E04FEF50E082279327A427B52721
:100750008093600090936100A0936200B093630067
:1007600008950E94A202EBE8F0E020E031E0C90128
:100770000296808391833396220F331F80E0EA39FB
:10078000F807A9F782E8808311820E94080280E8B6
:1007900085BF1BBA9FEF98BB8FE085BB92BB8FE1F3
:1007A0008ABB97BB94BB8AEF81BB85E687B987ED8F
:1007B00086B984E090E297BD86BD82E890E09BBD5B
:1007C0008ABD84E690E199BD88BD88E389BF89E14F
:1007D0008EBD0E94740188957720E9F70E9453032B
:1007E00088957720E9F3F7CF97FB092E07260AD0E3
:1007F00077FD04D00CD006D000201AF470956195D6
:100800007F4F0895F6F7909581959F4F0895AA1B05
:10081000BB1B51E107C0AA1FBB1FA617B70710F0EB
:10082000A61BB70B881F991F5A95A9F7809590951D
:0A083000BC01CD010895F894FFCF3C
:04083A0000F2FF00C9
:00000001FF
